:020000040000FA
:100000008E018F01900191019201013093009401C2
:100010008501860198018316860110308500043021
:1000200081008312051EDE284220842098080319CF
:100030001B28851598030B1D1B288B01B0200C086D
:10004000143A031D2528860185018C0B1B281428D2
:100050000F398207FC340234D134B134673496341A
:100060009E348034FF34F13400340F398207003479
:1000700001340134043400340234023405340034D1
:10008000063400347A308C008E0A0E08093C0318BE
:1000900008007B308C008E018F0A0F08053C031886
:1000A000080079308C008F01900A1008093C031871
:1000B00008007B308C009001910A1108053C031860
:1000C00008007C308C0091011308013C0318722851
:1000D000920A1208033C03187C287D308C009201A0
:1000E00093017C28920A1208093C03187C287D3071
:1000F0008C009201930A7C28120898009308031937
:1001000083280A30980708009501940A1408063CD1
:10011000031C94011408013A03199C28033A03199B
:10012000A128013A0319A428073A0319A728003087
:10013000860000308500080095151308031DA928C6
:10014000080015151208A92895141108A9281514D6
:100150001008970028208600170835208500080021
:10016000051A0800950803190800970A1708093CA2
:10017000031C97011708A920D620051EBD28D620EC
:10018000051EBD2814309600051EB528D620960BF6
:10019000C428170894018F018E0195199300151931
:1001A0009200951891001518900014280C308C00BE
:1001B0000B1DD8288B018C0BD82808009601160837
:1001C000A920D620D620960A16080A3A031DDF2851
:0201D000DE2827
:02400E00F13F80
:00000001FF
